 redefclass008

 Timestamp is 3c113f34 (reproducible build file hash)

 Preferred load address is 0000000180000000

 Start         Length     Name                   Class
 0001:00000000 00002ec0H .text$mn                CODE
 0001:00002ec0 00000036H .text$mn$00             CODE
 0001:00002ef6 00000092H .text$x                 CODE
 0002:00000000 00000190H .idata$5                DATA
 0002:00000190 00000038H .00cfg                  DATA
 0002:000001c8 00000008H .CRT$XCA                DATA
 0002:000001d0 00000008H .CRT$XCZ                DATA
 0002:000001d8 00000008H .CRT$XIA                DATA
 0002:000001e0 00000008H .CRT$XIC                DATA
 0002:000001e8 00000008H .CRT$XIZ                DATA
 0002:000001f0 00000008H .CRT$XLA                DATA
 0002:000001f8 00000008H .CRT$XLZ                DATA
 0002:00000200 00000008H .CRT$XPA                DATA
 0002:00000208 00000008H .CRT$XPZ                DATA
 0002:00000210 00000008H .CRT$XTA                DATA
 0002:00000218 00000008H .CRT$XTZ                DATA
 0002:00000220 00000000H .gehcont$y              DATA
 0002:00000220 00000000H .gfids$y                DATA
 0002:00000220 000020e0H .rdata                  DATA
 0002:00002300 00000000H .rdata$CastGuardVftablesA DATA
 0002:00002300 00000000H .rdata$CastGuardVftablesC DATA
 0002:00002300 00000028H .rdata$T                DATA
 0002:00002328 000000b0H .rdata$voltmd           DATA
 0002:000023d8 00000320H .rdata$zzzdbg           DATA
 0002:000026f8 00000008H .rtc$IAA                DATA
 0002:00002700 00000008H .rtc$IZZ                DATA
 0002:00002708 00000008H .rtc$TAA                DATA
 0002:00002710 00000008H .rtc$TZZ                DATA
 0002:00002718 00000004H .tls                    DATA
 0002:0000271c 00000004H .tls$                   DATA
 0002:00002720 00000008H .tls$ZZZ                DATA
 0002:00002728 00000318H .xdata                  DATA
 0002:00002a40 00000434H .edata                  DATA
 0002:00002e74 00000064H .idata$2                DATA
 0002:00002ed8 00000018H .idata$3                DATA
 0002:00002ef0 00000190H .idata$4                DATA
 0002:00003080 00000414H .idata$6                DATA
 0003:00000000 00000140H .data                   DATA
 0003:00000140 0001b388H .bss                    DATA
 0004:00000000 00000384H .pdata                  DATA

  Address         Publics by Value              Rva+Base               Lib:Object

 0000:00000000       __AbsoluteZero             0000000000000000     <absolute>
 0000:00000000       ___safe_se_handler_count   0000000000000000     <absolute>
 0000:00000000       ___safe_se_handler_table   0000000000000000     <absolute>
 0000:00000000       __arm64x_extra_rfe_table   0000000000000000     <absolute>
 0000:00000000       __arm64x_extra_rfe_table_size 0000000000000000     <absolute>
 0000:00000000       __arm64x_native_entrypoint 0000000000000000     <absolute>
 0000:00000000       __arm64x_redirection_metadata 0000000000000000     <absolute>
 0000:00000000       __arm64x_redirection_metadata_count 0000000000000000     <absolute>
 0000:00000000       __dynamic_value_reloc_table 0000000000000000     <absolute>
 0000:00000000       __enclave_config           0000000000000000     <absolute>
 0000:00000000       __guard_check_icall_a64n_fptr 0000000000000000     <absolute>
 0000:00000000       __guard_eh_cont_count      0000000000000000     <absolute>
 0000:00000000       __guard_eh_cont_table      0000000000000000     <absolute>
 0000:00000000       __guard_fids_count         0000000000000000     <absolute>
 0000:00000000       __guard_fids_table         0000000000000000     <absolute>
 0000:00000000       __guard_iat_count          0000000000000000     <absolute>
 0000:00000000       __guard_iat_table          0000000000000000     <absolute>
 0000:00000000       __guard_longjmp_count      0000000000000000     <absolute>
 0000:00000000       __guard_longjmp_table      0000000000000000     <absolute>
 0000:00000000       __hybrid_auxiliary_iat     0000000000000000     <absolute>
 0000:00000000       __hybrid_auxiliary_iat_copy 0000000000000000     <absolute>
 0000:00000000       __hybrid_code_map          0000000000000000     <absolute>
 0000:00000000       __hybrid_code_map_count    0000000000000000     <absolute>
 0000:00000000       __x64_code_ranges_to_entry_points 0000000000000000     <absolute>
 0000:00000000       __x64_code_ranges_to_entry_points_count 0000000000000000     <absolute>
 0000:00000100       __guard_flags              0000000000000100     <absolute>
 0000:00000000       __ImageBase                0000000180000000     <linker-defined>
 0001:00000000       ?NewObject@JNIEnv_@@QEAAPEAV_jobject@@PEAV_jclass@@PEAU_jmethodID@@ZZ 0000000180001000 f i libredefclass008.obj
 0001:00000024       ?SetEventNotificationMode@_jvmtiEnv@@QEAA?AW4jvmtiError@@W4jvmtiEventMode@@W4jvmtiEvent@@PEAV_jobject@@ZZ 0000000180001024 f i libredefclass008.obj
 0001:0000002c       ?TranslateError@@YAPEBDW4jvmtiError@@@Z 000000018000102c f   libredefclass008.obj
 0001:000002e4       ?nsk_jni_check_exception@@YAHPEAUJNIEnv_@@QEBDH@Z 00000001800012e4 f   libredefclass008.obj
 0001:00000428       ?nsk_jni_lverify@@YAHHPEAUJNIEnv_@@HQEBDH1ZZ 0000000180001428 f   libredefclass008.obj
 0001:000004c8       Agent_Initialize           00000001800014c8 f   libredefclass008.obj
 0001:00000624       Agent_OnAttach             0000000180001624 f   libredefclass008.obj
 0001:00000624       Agent_OnLoad               0000000180001624 f   libredefclass008.obj
 0001:0000062c       Breakpoint                 000000018000162c f   libredefclass008.obj
 0001:0000062c       _guard_check_icall_nop     000000018000162c f   MSVCRT:guard_support.obj
 0001:00000630       Java_nsk_jvmti_RedefineClasses_redefclass008_getResult 0000000180001630 f   libredefclass008.obj
 0001:0000083c       Java_nsk_jvmti_RedefineClasses_redefclass008_makeRedefinition 000000018000183c f   libredefclass008.obj
 0001:00000938       Java_nsk_jvmti_RedefineClasses_redefclass008_setBreakpoints 0000000180001938 f   libredefclass008.obj
 0001:00000b08       Java_nsk_jvmti_unit_FollowReferences_FollowRefObjects_addRefToVerify 0000000180001b08 f   libredefclass008.obj
 0001:00000cc4       Java_nsk_jvmti_unit_FollowReferences_FollowRefObjects_getTag 0000000180001cc4 f   libredefclass008.obj
 0001:00000d80       Java_nsk_jvmti_unit_FollowReferences_FollowRefObjects_resetRefsToVerify 0000000180001d80 f   libredefclass008.obj
 0001:00000d88       Java_nsk_jvmti_unit_FollowReferences_FollowRefObjects_resetTags 0000000180001d88 f   libredefclass008.obj
 0001:00000dcc       Java_nsk_jvmti_unit_FollowReferences_FollowRefObjects_setTag 0000000180001dcc f   libredefclass008.obj
 0001:00001018       Java_nsk_share_jvmti_ArgumentHandler_getAgentOptionsString 0000000180002018 f   libredefclass008.obj
 0001:000010c4       Java_nsk_share_jvmti_DebugeeClass_checkStatus 00000001800020c4 f   libredefclass008.obj
 0001:0000114c       Java_nsk_share_jvmti_DebugeeClass_resetAgentData 000000018000214c f   libredefclass008.obj
 0001:000011ac       Java_nsk_share_jvmti_RedefineAgent_agentStatus 00000001800021ac f   libredefclass008.obj
 0001:000011b8       Java_nsk_share_jvmti_RedefineAgent_isRedefined 00000001800021b8 f   libredefclass008.obj
 0001:000011c4       Java_nsk_share_jvmti_RedefineAgent_redefineAttempted 00000001800021c4 f   libredefclass008.obj
 0001:000011d0       MA_checkStatus             00000001800021d0 f   libredefclass008.obj
 0001:00001274       __local_stdio_printf_options 0000000180002274 f i libredefclass008.obj
 0001:00001444       exitOnError                0000000180002444 f   libredefclass008.obj
 0001:000014f8       fprintf                    00000001800024f8 f i libredefclass008.obj
 0001:0000153c       nsk_jvmti_lverify          000000018000253c f   libredefclass008.obj
 0001:0000162c       nsk_jvmti_resetAgentData   000000018000262c f   libredefclass008.obj
 0001:000016a0       nsk_lcomplain              00000001800026a0 f   libredefclass008.obj
 0001:000016c0       nsk_ldisplay               00000001800026c0 f   libredefclass008.obj
 0001:000016e0       nsk_ltrace                 00000001800026e0 f   libredefclass008.obj
 0001:00001700       nsk_lvcomplain             0000000180002700 f   libredefclass008.obj
 0001:000018b8       nsk_lvdisplay              00000001800028b8 f   libredefclass008.obj
 0001:00001904       nsk_lverify                0000000180002904 f   libredefclass008.obj
 0001:00001960       nsk_lvtrace                0000000180002960 f   libredefclass008.obj
 0001:000019c0       nsk_printf                 00000001800029c0 f   libredefclass008.obj
 0001:000019e8       nsk_vprintf                00000001800029e8 f   libredefclass008.obj
 0001:00001a9c       printf                     0000000180002a9c f i libredefclass008.obj
 0001:00001f9c       __raise_securityfailure    0000000180002f9c f   MSVCRT:gs_report.obj
 0001:00001fd0       __report_gsfailure         0000000180002fd0 f   MSVCRT:gs_report.obj
 0001:00002210       __GSHandlerCheck           0000000180003210 f   MSVCRT:gshandler.obj
 0001:00002230       __GSHandlerCheckCommon     0000000180003230 f   MSVCRT:gshandler.obj
 0001:000022a0       __security_check_cookie    00000001800032a0 f   MSVCRT:amdsecgs.obj
 0001:000025e0       _DllMainCRTStartup         00000001800035e0 f   MSVCRT:dll_dllmain.obj
 0001:00002620       __scrt_acquire_startup_lock 0000000180003620 f   MSVCRT:utility.obj
 0001:0000265c       __scrt_dllmain_after_initialize_c 000000018000365c f   MSVCRT:utility.obj
 0001:00002690       __scrt_dllmain_before_initialize_c 0000000180003690 f   MSVCRT:utility.obj
 0001:000026a8       __scrt_dllmain_crt_thread_attach 00000001800036a8 f   MSVCRT:utility.obj
 0001:000026d0       __scrt_dllmain_crt_thread_detach 00000001800036d0 f   MSVCRT:utility.obj
 0001:000026e8       __scrt_dllmain_exception_filter 00000001800036e8 f   MSVCRT:utility.obj
 0001:00002748       __scrt_dllmain_uninitialize_c 0000000180003748 f   MSVCRT:utility.obj
 0001:00002778       __scrt_dllmain_uninitialize_critical 0000000180003778 f   MSVCRT:utility.obj
 0001:0000278c       __scrt_initialize_crt      000000018000378c f   MSVCRT:utility.obj
 0001:000027d8       __scrt_initialize_onexit_tables 00000001800037d8 f   MSVCRT:utility.obj
 0001:00002864       __scrt_is_nonwritable_in_current_image 0000000180003864 f   MSVCRT:utility.obj
 0001:000028fc       __scrt_release_startup_lock 00000001800038fc f   MSVCRT:utility.obj
 0001:00002920       __scrt_uninitialize_crt    0000000180003920 f   MSVCRT:utility.obj
 0001:0000294c       _onexit                    000000018000394c f   MSVCRT:utility.obj
 0001:00002988       atexit                     0000000180003988 f   MSVCRT:utility.obj
 0001:000029a0       __crt_debugger_hook        00000001800039a0 f   MSVCRT:utility_desktop.obj
 0001:000029a8       __scrt_fastfail            00000001800039a8 f   MSVCRT:utility_desktop.obj
 0001:00002af4       __security_init_cookie     0000000180003af4 f   MSVCRT:gs_support.obj
 0001:00002ba0       DllMain                    0000000180003ba0 f   MSVCRT:dll_dllmain_stub.obj
 0001:00002bc4       ?__scrt_initialize_type_info@@YAXXZ 0000000180003bc4 f   MSVCRT:tncleanup.obj
 0001:00002bd4       ?__scrt_uninitialize_type_info@@YAXXZ 0000000180003bd4 f   MSVCRT:tncleanup.obj
 0001:00002be0       __local_stdio_scanf_options 0000000180003be0 f i MSVCRT:default_local_stdio_options.obj
 0001:00002be8       __scrt_initialize_default_local_stdio_options 0000000180003be8 f   MSVCRT:default_local_stdio_options.obj
 0001:00002c04       __scrt_get_dyn_tls_init_callback 0000000180003c04 f   MSVCRT:dyn_tls_init.obj
 0001:00002c0c       _RTC_Initialize            0000000180003c0c f   MSVCRT:initsect.obj
 0001:00002c48       _RTC_Terminate             0000000180003c48 f   MSVCRT:initsect.obj
 0001:00002c84       __isa_available_init       0000000180003c84 f   MSVCRT:cpu_disp.obj
 0001:00002e30       _get_startup_argv_mode     0000000180003e30 f   MSVCRT:argv_mode.obj
 0001:00002e38       __scrt_is_ucrt_dll_in_use  0000000180003e38 f   MSVCRT:ucrt_detection.obj
 0001:00002e50       memcpy                     0000000180003e50 f   vcruntime:VCRUNTIME140.dll
 0001:00002e56       memset                     0000000180003e56 f   vcruntime:VCRUNTIME140.dll
 0001:00002e5c       strchr                     0000000180003e5c f   vcruntime:VCRUNTIME140.dll
 0001:00002e62       __C_specific_handler       0000000180003e62 f   vcruntime:VCRUNTIME140.dll
 0001:00002e68       __std_type_info_destroy_list 0000000180003e68 f   vcruntime:VCRUNTIME140.dll
 0001:00002e6e       strlen                     0000000180003e6e f   ucrt:api-ms-win-crt-string-l1-1-0.dll
 0001:00002e74       _initterm                  0000000180003e74 f   ucrt:api-ms-win-crt-runtime-l1-1-0.dll
 0001:00002e7a       _initterm_e                0000000180003e7a f   ucrt:api-ms-win-crt-runtime-l1-1-0.dll
 0001:00002e80       _seh_filter_dll            0000000180003e80 f   ucrt:api-ms-win-crt-runtime-l1-1-0.dll
 0001:00002e86       _configure_narrow_argv     0000000180003e86 f   ucrt:api-ms-win-crt-runtime-l1-1-0.dll
 0001:00002e8c       _initialize_narrow_environment 0000000180003e8c f   ucrt:api-ms-win-crt-runtime-l1-1-0.dll
 0001:00002e92       _initialize_onexit_table   0000000180003e92 f   ucrt:api-ms-win-crt-runtime-l1-1-0.dll
 0001:00002e98       _register_onexit_function  0000000180003e98 f   ucrt:api-ms-win-crt-runtime-l1-1-0.dll
 0001:00002e9e       _execute_onexit_table      0000000180003e9e f   ucrt:api-ms-win-crt-runtime-l1-1-0.dll
 0001:00002ea4       _crt_atexit                0000000180003ea4 f   ucrt:api-ms-win-crt-runtime-l1-1-0.dll
 0001:00002eaa       _cexit                     0000000180003eaa f   ucrt:api-ms-win-crt-runtime-l1-1-0.dll
 0001:00002eb0       __acrt_initialize          0000000180003eb0 f   MSVCRT:ucrt_stubs.obj
 0001:00002eb0       __acrt_thread_attach       0000000180003eb0 f   MSVCRT:ucrt_stubs.obj
 0001:00002eb0       __acrt_thread_detach       0000000180003eb0 f   MSVCRT:ucrt_stubs.obj
 0001:00002eb0       __acrt_uninitialize        0000000180003eb0 f   MSVCRT:ucrt_stubs.obj
 0001:00002eb0       __acrt_uninitialize_critical 0000000180003eb0 f   MSVCRT:ucrt_stubs.obj
 0001:00002eb0       __scrt_stub_for_acrt_initialize 0000000180003eb0 f   MSVCRT:ucrt_stubs.obj
 0001:00002eb0       __scrt_stub_for_acrt_thread_attach 0000000180003eb0 f   MSVCRT:ucrt_stubs.obj
 0001:00002eb0       __scrt_stub_for_acrt_thread_detach 0000000180003eb0 f   MSVCRT:ucrt_stubs.obj
 0001:00002eb0       __scrt_stub_for_acrt_uninitialize 0000000180003eb0 f   MSVCRT:ucrt_stubs.obj
 0001:00002eb0       __scrt_stub_for_acrt_uninitialize_critical 0000000180003eb0 f   MSVCRT:ucrt_stubs.obj
 0001:00002eb0       __vcrt_initialize          0000000180003eb0 f   MSVCRT:ucrt_stubs.obj
 0001:00002eb0       __vcrt_thread_attach       0000000180003eb0 f   MSVCRT:ucrt_stubs.obj
 0001:00002eb0       __vcrt_thread_detach       0000000180003eb0 f   MSVCRT:ucrt_stubs.obj
 0001:00002eb0       __vcrt_uninitialize        0000000180003eb0 f   MSVCRT:ucrt_stubs.obj
 0001:00002eb0       __vcrt_uninitialize_critical 0000000180003eb0 f   MSVCRT:ucrt_stubs.obj
 0001:00002eb4       __scrt_stub_for_is_c_termination_complete 0000000180003eb4 f   MSVCRT:ucrt_stubs.obj
 0001:00002eb4       _is_c_termination_complete 0000000180003eb4 f   MSVCRT:ucrt_stubs.obj
 0001:00002ed0       _guard_dispatch_icall_nop  0000000180003ed0 f   MSVCRT:guard_dispatch.obj
 0001:00002ef0       _guard_xfg_dispatch_icall_nop 0000000180003ef0 f   MSVCRT:guard_xfg_dispatch.obj
 0002:00000000       __imp_RtlCaptureContext    0000000180004000     kernel32:KERNEL32.dll
 0002:00000008       __imp_RtlLookupFunctionEntry 0000000180004008     kernel32:KERNEL32.dll
 0002:00000010       __imp_RtlVirtualUnwind     0000000180004010     kernel32:KERNEL32.dll
 0002:00000018       __imp_UnhandledExceptionFilter 0000000180004018     kernel32:KERNEL32.dll
 0002:00000020       __imp_SetUnhandledExceptionFilter 0000000180004020     kernel32:KERNEL32.dll
 0002:00000028       __imp_GetCurrentProcess    0000000180004028     kernel32:KERNEL32.dll
 0002:00000030       __imp_TerminateProcess     0000000180004030     kernel32:KERNEL32.dll
 0002:00000038       __imp_IsProcessorFeaturePresent 0000000180004038     kernel32:KERNEL32.dll
 0002:00000040       __imp_CloseHandle          0000000180004040     kernel32:KERNEL32.dll
 0002:00000048       __imp_InitializeCriticalSectionAndSpinCount 0000000180004048     kernel32:KERNEL32.dll
 0002:00000050       __imp_DeleteCriticalSection 0000000180004050     kernel32:KERNEL32.dll
 0002:00000058       __imp_CreateEventW         0000000180004058     kernel32:KERNEL32.dll
 0002:00000060       __imp_GetModuleHandleW     0000000180004060     kernel32:KERNEL32.dll
 0002:00000068       __imp_GetProcAddress       0000000180004068     kernel32:KERNEL32.dll
 0002:00000070       __imp_IsDebuggerPresent    0000000180004070     kernel32:KERNEL32.dll
 0002:00000078       __imp_QueryPerformanceCounter 0000000180004078     kernel32:KERNEL32.dll
 0002:00000080       __imp_GetCurrentProcessId  0000000180004080     kernel32:KERNEL32.dll
 0002:00000088       __imp_GetCurrentThreadId   0000000180004088     kernel32:KERNEL32.dll
 0002:00000090       __imp_GetSystemTimeAsFileTime 0000000180004090     kernel32:KERNEL32.dll
 0002:00000098       __imp_DisableThreadLibraryCalls 0000000180004098     kernel32:KERNEL32.dll
 0002:000000a0       __imp_InitializeSListHead  00000001800040a0     kernel32:KERNEL32.dll
 0002:000000a8       \177KERNEL32_NULL_THUNK_DATA 00000001800040a8     kernel32:KERNEL32.dll
 0002:000000b0       __imp_memcpy               00000001800040b0     vcruntime:VCRUNTIME140.dll
 0002:000000b8       __imp_memset               00000001800040b8     vcruntime:VCRUNTIME140.dll
 0002:000000c0       __imp_strchr               00000001800040c0     vcruntime:VCRUNTIME140.dll
 0002:000000c8       __imp___C_specific_handler 00000001800040c8     vcruntime:VCRUNTIME140.dll
 0002:000000d0       __imp___std_type_info_destroy_list 00000001800040d0     vcruntime:VCRUNTIME140.dll
 0002:000000d8       \177VCRUNTIME140_NULL_THUNK_DATA 00000001800040d8     vcruntime:VCRUNTIME140.dll
 0002:000000e0       __imp__errno               00000001800040e0     ucrt:api-ms-win-crt-runtime-l1-1-0.dll
 0002:000000e8       __imp_exit                 00000001800040e8     ucrt:api-ms-win-crt-runtime-l1-1-0.dll
 0002:000000f0       __imp__cexit               00000001800040f0     ucrt:api-ms-win-crt-runtime-l1-1-0.dll
 0002:000000f8       __imp__crt_atexit          00000001800040f8     ucrt:api-ms-win-crt-runtime-l1-1-0.dll
 0002:00000100       __imp__execute_onexit_table 0000000180004100     ucrt:api-ms-win-crt-runtime-l1-1-0.dll
 0002:00000108       __imp__register_onexit_function 0000000180004108     ucrt:api-ms-win-crt-runtime-l1-1-0.dll
 0002:00000110       __imp__initialize_onexit_table 0000000180004110     ucrt:api-ms-win-crt-runtime-l1-1-0.dll
 0002:00000118       __imp__initialize_narrow_environment 0000000180004118     ucrt:api-ms-win-crt-runtime-l1-1-0.dll
 0002:00000120       __imp__configure_narrow_argv 0000000180004120     ucrt:api-ms-win-crt-runtime-l1-1-0.dll
 0002:00000128       __imp__seh_filter_dll      0000000180004128     ucrt:api-ms-win-crt-runtime-l1-1-0.dll
 0002:00000130       __imp__initterm_e          0000000180004130     ucrt:api-ms-win-crt-runtime-l1-1-0.dll
 0002:00000138       __imp__initterm            0000000180004138     ucrt:api-ms-win-crt-runtime-l1-1-0.dll
 0002:00000140       \177api-ms-win-crt-runtime-l1-1-0_NULL_THUNK_DATA 0000000180004140     ucrt:api-ms-win-crt-runtime-l1-1-0.dll
 0002:00000148       __imp___acrt_iob_func      0000000180004148     ucrt:api-ms-win-crt-stdio-l1-1-0.dll
 0002:00000150       __imp_fflush               0000000180004150     ucrt:api-ms-win-crt-stdio-l1-1-0.dll
 0002:00000158       __imp___stdio_common_vsprintf 0000000180004158     ucrt:api-ms-win-crt-stdio-l1-1-0.dll
 0002:00000160       __imp___stdio_common_vfprintf 0000000180004160     ucrt:api-ms-win-crt-stdio-l1-1-0.dll
 0002:00000168       \177api-ms-win-crt-stdio-l1-1-0_NULL_THUNK_DATA 0000000180004168     ucrt:api-ms-win-crt-stdio-l1-1-0.dll
 0002:00000170       __imp__strdup              0000000180004170     ucrt:api-ms-win-crt-string-l1-1-0.dll
 0002:00000170       __imp_strdup               0000000180004170     ucrt:api-ms-win-crt-string-l1-1-0.dll
 0002:00000178       __imp_strlen               0000000180004178     ucrt:api-ms-win-crt-string-l1-1-0.dll
 0002:00000180       __imp_strncpy              0000000180004180     ucrt:api-ms-win-crt-string-l1-1-0.dll
 0002:00000188       \177api-ms-win-crt-string-l1-1-0_NULL_THUNK_DATA 0000000180004188     ucrt:api-ms-win-crt-string-l1-1-0.dll
 0002:00000190       __guard_check_icall_fptr   0000000180004190     MSVCRT:guard_support.obj
 0002:00000198       __guard_xfg_check_icall_fptr 0000000180004198     MSVCRT:guard_support.obj
 0002:000001a0       __guard_dispatch_icall_fptr 00000001800041a0     MSVCRT:guard_support.obj
 0002:000001a8       __guard_xfg_dispatch_icall_fptr 00000001800041a8     MSVCRT:guard_support.obj
 0002:000001b0       __guard_xfg_table_dispatch_icall_fptr 00000001800041b0     MSVCRT:guard_support.obj
 0002:000001b8       __castguard_check_failure_os_handled_fptr 00000001800041b8     MSVCRT:guard_support.obj
 0002:000001c0       __guard_memcpy_fptr        00000001800041c0     vcruntime:softmemtag.obj
 0002:000001c8       __xc_a                     00000001800041c8     MSVCRT:initializers.obj
 0002:000001d0       __xc_z                     00000001800041d0     MSVCRT:initializers.obj
 0002:000001d8       __xi_a                     00000001800041d8     MSVCRT:initializers.obj
 0002:000001e8       __xi_z                     00000001800041e8     MSVCRT:initializers.obj
 0002:000001f0       __xl_a                     00000001800041f0     MSVCRT:tlssup.obj
 0002:000001f8       __xl_z                     00000001800041f8     MSVCRT:tlssup.obj
 0002:00000200       __xp_a                     0000000180004200     MSVCRT:initializers.obj
 0002:00000208       __xp_z                     0000000180004208     MSVCRT:initializers.obj
 0002:00000210       __xt_a                     0000000180004210     MSVCRT:initializers.obj
 0002:00000218       __xt_z                     0000000180004218     MSVCRT:initializers.obj
 0002:00000220       g_refKindStr               0000000180004220     libredefclass008.obj
 0002:000003d0       ??_C@_09BPLDFGCI@unknown_0@ 00000001800043d0     libredefclass008.obj
 0002:000003e0       ??_C@_0BL@FPNMECJD@JVMTI_HEAP_REFERENCE_CLASS@ 00000001800043e0     libredefclass008.obj
 0002:00000400       ??_C@_0BL@FKGKKLNM@JVMTI_HEAP_REFERENCE_FIELD@ 0000000180004400     libredefclass008.obj
 0002:00000420       ??_C@_0CD@CAEHCFJF@JVMTI_HEAP_REFERENCE_ARRAY_ELEM@ 0000000180004420     libredefclass008.obj
 0002:00000448       ??_C@_0CC@DNEBMCNK@JVMTI_HEAP_REFERENCE_CLASS_LOAD@ 0000000180004448     libredefclass008.obj
 0002:00000470       ??_C@_0BN@CJMIPEBB@JVMTI_HEAP_REFERENCE_SIGNERS@ 0000000180004470     libredefclass008.obj
 0002:00000490       ??_C@_0CH@HBOIDPEB@JVMTI_HEAP_REFERENCE_PROTECTION@ 0000000180004490     libredefclass008.obj
 0002:000004b8       ??_C@_0BP@MDKGDGKL@JVMTI_HEAP_REFERENCE_INTERFACE@ 00000001800044b8     libredefclass008.obj
 0002:000004d8       ??_C@_0CC@JJMIHNJH@JVMTI_HEAP_REFERENCE_STATIC_FIE@ 00000001800044d8     libredefclass008.obj
 0002:00000500       ??_C@_0CD@IDHEEGID@JVMTI_HEAP_REFERENCE_CONSTANT_P@ 0000000180004500     libredefclass008.obj
 0002:00000528       ??_C@_0CA@EFFCHNG@JVMTI_HEAP_REFERENCE_SUPERCLASS@ 0000000180004528     libredefclass008.obj
 0002:00000548       ??_C@_0L@PCDFHGCJ@unknown_11@ 0000000180004548     libredefclass008.obj
 0002:00000558       ??_C@_0L@NJBICFOK@unknown_12@ 0000000180004558     libredefclass008.obj
 0002:00000568       ??_C@_0L@MAADBEKL@unknown_13@ 0000000180004568     libredefclass008.obj
 0002:00000578       ??_C@_0L@IPECICGM@unknown_14@ 0000000180004578     libredefclass008.obj
 0002:00000588       ??_C@_0L@JGFJLDCN@unknown_15@ 0000000180004588     libredefclass008.obj
 0002:00000598       ??_C@_0L@LNHEOAOO@unknown_16@ 0000000180004598     libredefclass008.obj
 0002:000005a8       ??_C@_0L@KEGPNBKP@unknown_17@ 00000001800045a8     libredefclass008.obj
 0002:000005b8       ??_C@_0L@CDPHMNGA@unknown_18@ 00000001800045b8     libredefclass008.obj
 0002:000005c8       ??_C@_0L@DKOMPMCB@unknown_19@ 00000001800045c8     libredefclass008.obj
 0002:000005d8       ??_C@_0L@OJGIPJDB@unknown_20@ 00000001800045d8     libredefclass008.obj
 0002:000005e8       ??_C@_0CA@KAOFNDEM@JVMTI_HEAP_REFERENCE_JNI_GLOBAL@ 00000001800045e8     libredefclass008.obj
 0002:00000608       ??_C@_0CC@HPFAJBK@JVMTI_HEAP_REFERENCE_SYSTEM_CLA@ 0000000180004608     libredefclass008.obj
 0002:00000630       ??_C@_0BN@FDEGFOHC@JVMTI_HEAP_REFERENCE_MONITOR@ 0000000180004630     libredefclass008.obj
 0002:00000650       ??_C@_0CB@HKIBCMAJ@JVMTI_HEAP_REFERENCE_STACK_LOCA@ 0000000180004650     libredefclass008.obj
 0002:00000678       ??_C@_0BP@EAACMMOE@JVMTI_HEAP_REFERENCE_JNI_LOCAL@ 0000000180004678     libredefclass008.obj
 0002:00000698       ??_C@_0BM@IJDEOGOE@JVMTI_HEAP_REFERENCE_THREAD@ 0000000180004698     libredefclass008.obj
 0002:000006b8       ??_C@_0BL@EDGPPKC@JVMTI_HEAP_REFERENCE_OTHER@ 00000001800046b8     libredefclass008.obj
 0002:000006d4       ??_C@_04BCJPDBDA@Code@     00000001800046d4     libredefclass008.obj
 0002:000006e0       ??_C@_0BA@OCLMCFKC@LineNumberTable@ 00000001800046e0     libredefclass008.obj
 0002:000006f0       ??_C@_0BD@CPAEPILC@LocalVariableTable@ 00000001800046f0     libredefclass008.obj
 0002:00000708       ??_C@_0BH@NMBDNHBD@LocalVariableTypeTable@ 0000000180004708     libredefclass008.obj
 0002:00000720       ??_C@_0O@HIHEEDNJ@StackMapTable@ 0000000180004720     libredefclass008.obj
 0002:00000730       ??_C@_07CCHEGMIH@checkIt@  0000000180004730     libredefclass008.obj
 0002:00000738       ??_C@_0BK@NEDFEFGA@?$CILjava?1io?1PrintStream?$DLZ?$CJI@ 0000000180004738     libredefclass008.obj
 0002:00000758       ??_C@_09DIBCFHMF@finMethod@ 0000000180004758     libredefclass008.obj
 0002:00000764       ??_C@_06EKDFHLKM@?$CIJIJ?$CJV@ 0000000180004764     libredefclass008.obj
 0002:00000770       ??_C@_0L@KCCHGEID@statMethod@ 0000000180004770     libredefclass008.obj
 0002:0000077c       ??_C@_06BDEOKIHC@?$CIIII?$CJI@ 000000018000477c     libredefclass008.obj
 0002:00000788       ??_C@_0L@HCDIAMJG@?9?5?$CFs?0?5?$CFd?3?5@ 0000000180004788     libredefclass008.obj
 0002:000007a0       ??_C@_0JI@HLPECLFI@?$CD?5?4?4?4?6?$CD?5ERROR?3?5too?5many?5complai@ 00000001800047a0     libredefclass008.obj
 0002:00000840       ??_C@_0ED@JNEKCCOB@The?5following?5fake?5exception?5st@ 0000000180004840     libredefclass008.obj
 0002:00000888       ??_C@_0CN@FCNMDFBH@nsk?4share?4Fake_Exception_for_RU@ 0000000180004888     libredefclass008.obj
 0002:000008b8       ??_C@_08PGFFNAEI@?$CI?$CFs?3?$CFd?$CJ?5@ 00000001800048b8     libredefclass008.obj
 0002:000008c8       ??_C@_0DP@IENMAEGI@s?2test?2hotspot?2jtreg?2vmTestbase@ 00000001800048c8     libredefclass008.obj
 0002:00000908       ??_C@_0BL@NDJLFFJB@?7at?5nsk_lvcomplain?$CI?$CFs?3?$CFd?$CJ?6@ 0000000180004908     libredefclass008.obj
 0002:00000928       ??_C@_0BC@JOOKAFKF@?$CD?5ERROR?3?5?$CFs?0?5?$CFd?3?5@ 0000000180004928     libredefclass008.obj
 0002:00000940       ??_C@_09KJEAHMEH@?$CD?5ERROR?3?5@ 0000000180004940     libredefclass008.obj
 0002:0000094c       ??_C@_02GPIOPFAK@?$DO?$DO@ 000000018000494c     libredefclass008.obj
 0002:00000950       ??_C@_02FODMEDOG@?$DM?$DM@ 0000000180004950     libredefclass008.obj
 0002:00000954       ??_C@_02DJGKEECL@?4?4@     0000000180004954     libredefclass008.obj
 0002:00000958       ??_C@_0O@CJPGJOAF@?9?5?$CFs?0?5?$CFd?3?5?$CFs?5@ 0000000180004958     libredefclass008.obj
 0002:00000968       ??_C@_0CB@IAKPDOIC@?$CD?5?5?5verified?5assertion?5is?5FALSE@ 0000000180004968     libredefclass008.obj
 0002:00000990       ??_C@_0CO@LGONDEPD@stdout?3?5fflush?5failed?5?9?5err?$DN?$CFd?5@ 0000000180004990     libredefclass008.obj
 0002:000009c0       ??_C@_0CO@KBGKJPBD@stderr?3?5fflush?5failed?5?9?5err?$DN?$CFd?5@ 00000001800049c0     libredefclass008.obj
 0002:000009f0       ??_C@_0BB@JCNMKLLK@JVMTI_ERROR_NONE@ 00000001800049f0     libredefclass008.obj
 0002:00000a08       ??_C@_0BL@LDIMKLPH@JVMTI_ERROR_INVALID_THREAD@ 0000000180004a08     libredefclass008.obj
 0002:00000a28       ??_C@_0CB@PJFPAIKJ@JVMTI_ERROR_INVALID_THREAD_GROU@ 0000000180004a28     libredefclass008.obj
 0002:00000a50       ??_C@_0BN@LLMKHMNF@JVMTI_ERROR_INVALID_PRIORITY@ 0000000180004a50     libredefclass008.obj
 0002:00000a70       ??_C@_0CB@MBOFKAGB@JVMTI_ERROR_THREAD_NOT_SUSPENDE@ 0000000180004a70     libredefclass008.obj
 0002:00000a98       ??_C@_0BN@FABOLPBI@JVMTI_ERROR_THREAD_SUSPENDED@ 0000000180004a98     libredefclass008.obj
 0002:00000ab8       ??_C@_0BN@FDGNOBJM@JVMTI_ERROR_THREAD_NOT_ALIVE@ 0000000180004ab8     libredefclass008.obj
 0002:00000ad8       ??_C@_0BL@GOBIFKNJ@JVMTI_ERROR_INVALID_OBJECT@ 0000000180004ad8     libredefclass008.obj
 0002:00000af8       ??_C@_0BK@FCMAJPPC@JVMTI_ERROR_INVALID_CLASS@ 0000000180004af8     libredefclass008.obj
 0002:00000b18       ??_C@_0BP@IKLLBKEB@JVMTI_ERROR_CLASS_NOT_PREPARED@ 0000000180004b18     libredefclass008.obj
 0002:00000b38       ??_C@_0BN@KLPPLKG@JVMTI_ERROR_INVALID_METHODID@ 0000000180004b38     libredefclass008.obj
 0002:00000b58       ??_C@_0BN@BCEKOKND@JVMTI_ERROR_INVALID_LOCATION@ 0000000180004b58     libredefclass008.obj
 0002:00000b78       ??_C@_0BM@DFDGPME@JVMTI_ERROR_INVALID_FIELDID@ 0000000180004b78     libredefclass008.obj
 0002:00000b98       ??_C@_0BL@NELIEPEC@JVMTI_ERROR_NO_MORE_FRAMES@ 0000000180004b98     libredefclass008.obj
 0002:00000bb8       ??_C@_0BJ@BDBECFDM@JVMTI_ERROR_OPAQUE_FRAME@ 0000000180004bb8     libredefclass008.obj
 0002:00000bd8       ??_C@_0BK@MIIFNLOB@JVMTI_ERROR_TYPE_MISMATCH@ 0000000180004bd8     libredefclass008.obj
 0002:00000bf8       ??_C@_0BJ@HPCAOILC@JVMTI_ERROR_INVALID_SLOT@ 0000000180004bf8     libredefclass008.obj
 0002:00000c18       ??_C@_0BG@CHILOPNI@JVMTI_ERROR_DUPLICATE@ 0000000180004c18     libredefclass008.obj
 0002:00000c30       ??_C@_0BG@DIEMLHKM@JVMTI_ERROR_NOT_FOUND@ 0000000180004c30     libredefclass008.obj
 0002:00000c48       ??_C@_0BM@NHMCKHOB@JVMTI_ERROR_INVALID_MONITOR@ 0000000180004c48     libredefclass008.obj
 0002:00000c68       ??_C@_0BO@PPEDAJGL@JVMTI_ERROR_NOT_MONITOR_OWNER@ 0000000180004c68     libredefclass008.obj
 0002:00000c88       ??_C@_0BG@FCAIPEID@JVMTI_ERROR_INTERRUPT@ 0000000180004c88     libredefclass008.obj
 0002:00000ca0       ??_C@_0CB@EGDBNKOI@JVMTI_ERROR_INVALID_CLASS_FORMA@ 0000000180004ca0     libredefclass008.obj
 0002:00000cc8       ??_C@_0CG@DGKOGIAL@JVMTI_ERROR_CIRCULAR_CLASS_DEFI@ 0000000180004cc8     libredefclass008.obj
 0002:00000cf0       ??_C@_0BP@ICEALPKC@JVMTI_ERROR_FAILS_VERIFICATION@ 0000000180004cf0     libredefclass008.obj
 0002:00000d10       ??_C@_0DC@JDACLMIO@JVMTI_ERROR_UNSUPPORTED_REDEFIN@ 0000000180004d10     libredefclass008.obj
 0002:00000d48       ??_C@_0DE@GKDKNOMJ@JVMTI_ERROR_UNSUPPORTED_REDEFIN@ 0000000180004d48     libredefclass008.obj
 0002:00000d80       ??_C@_0BO@LAFKIOG@JVMTI_ERROR_INVALID_TYPESTATE@ 0000000180004d80     libredefclass008.obj
 0002:00000da0       ??_C@_0DH@INDGCLLB@JVMTI_ERROR_UNSUPPORTED_REDEFIN@ 0000000180004da0     libredefclass008.obj
 0002:00000dd8       ??_C@_0DE@NHEOMMGI@JVMTI_ERROR_UNSUPPORTED_REDEFIN@ 0000000180004dd8     libredefclass008.obj
 0002:00000e10       ??_C@_0CA@EKPNJOEP@JVMTI_ERROR_UNSUPPORTED_VERSION@ 0000000180004e10     libredefclass008.obj
 0002:00000e30       ??_C@_0BN@OFFMAHHL@JVMTI_ERROR_NAMES_DONT_MATCH@ 0000000180004e30     libredefclass008.obj
 0002:00000e50       ??_C@_0DN@HHBBLAKE@JVMTI_ERROR_UNSUPPORTED_REDEFIN@ 0000000180004e50     libredefclass008.obj
 0002:00000e90       ??_C@_0DO@HMBGBGNA@JVMTI_ERROR_UNSUPPORTED_REDEFIN@ 0000000180004e90     libredefclass008.obj
 0002:00000ed0       ??_C@_0BP@PBECGKHJ@JVMTI_ERROR_UNMODIFIABLE_CLASS@ 0000000180004ed0     libredefclass008.obj
 0002:00000ef0       ??_C@_0BK@CANILEHF@JVMTI_ERROR_NOT_AVAILABLE@ 0000000180004ef0     libredefclass008.obj
 0002:00000f10       ??_C@_0CE@INJKMEFK@JVMTI_ERROR_MUST_POSSESS_CAPABI@ 0000000180004f10     libredefclass008.obj
 0002:00000f38       ??_C@_0BJ@LBFPFPDM@JVMTI_ERROR_NULL_POINTER@ 0000000180004f38     libredefclass008.obj
 0002:00000f58       ??_C@_0BP@CHJPNNEM@JVMTI_ERROR_ABSENT_INFORMATION@ 0000000180004f58     libredefclass008.obj
 0002:00000f78       ??_C@_0BP@OMFMNLC@JVMTI_ERROR_INVALID_EVENT_TYPE@ 0000000180004f78     libredefclass008.obj
 0002:00000f98       ??_C@_0BN@BIBNPHHO@JVMTI_ERROR_ILLEGAL_ARGUMENT@ 0000000180004f98     libredefclass008.obj
 0002:00000fb8       ??_C@_0BK@KKNDHDCE@JVMTI_ERROR_NATIVE_METHOD@ 0000000180004fb8     libredefclass008.obj
 0002:00000fd8       ??_C@_0BK@PMKCFHAE@JVMTI_ERROR_OUT_OF_MEMORY@ 0000000180004fd8     libredefclass008.obj
 0002:00000ff8       ??_C@_0BK@NNJBDMNB@JVMTI_ERROR_ACCESS_DENIED@ 0000000180004ff8     libredefclass008.obj
 0002:00001018       ??_C@_0BI@GHECLMNC@JVMTI_ERROR_WRONG_PHASE@ 0000000180005018     libredefclass008.obj
 0002:00001030       ??_C@_0BF@OLIHJOII@JVMTI_ERROR_INTERNAL@ 0000000180005030     libredefclass008.obj
 0002:00001048       ??_C@_0BO@EOHGKJHI@JVMTI_ERROR_UNATTACHED_THREAD@ 0000000180005048     libredefclass008.obj
 0002:00001068       ??_C@_0CA@LKHFDACL@JVMTI_ERROR_INVALID_ENVIRONMENT@ 0000000180005068     libredefclass008.obj
 0002:00001088       ??_C@_0BA@MMFHLOKK@?$DMunknown?5error?$DO@ 0000000180005088     libredefclass008.obj
 0002:00001098       ??_C@_0CF@CBHOKDB@throwable?5?$DN?5jni?9?$DOExceptionOccur@ 0000000180005098     libredefclass008.obj
 0002:000010c0       ??_C@_03OFAPEBGM@?$CFs?6@  00000001800050c0     libredefclass008.obj
 0002:000010c8       ??_C@_0DM@LPIGEGNJ@s?2test?2hotspot?2jtreg?2vmTestbase@ 00000001800050c8     libredefclass008.obj
 0002:00001108       ??_C@_0CC@NFCNPEPK@Exception?5in?5JNI?5call?5?$CIcleared?$CJ@ 0000000180005108     libredefclass008.obj
 0002:00001130       ??_C@_0BJ@IBAKFIKF@jni?9?$DOExceptionDescribe?$CI?$CJ@ 0000000180005130     libredefclass008.obj
 0002:00001150       ??_C@_0BG@GGKALKMH@jni?9?$DOExceptionClear?$CI?$CJ@ 0000000180005150     libredefclass008.obj
 0002:00001168       ??_C@_0CF@JMGFGJLJ@?$CD?5?5?5verified?5JNI?5assertion?5is?5F@ 0000000180005168     libredefclass008.obj
 0002:00001190       ??_C@_0CB@MLNJNCLJ@?5?5jvmti?5error?3?5code?$DN?$CFd?0?5name?$DN?$CFs@ 0000000180005190     libredefclass008.obj
 0002:000011b8       ??_C@_0CD@OHBGDKMK@?$CD?5?5?5jvmti?5error?3?5code?$DN?$CFd?0?5name?$DN@ 00000001800051b8     libredefclass008.obj
 0002:000011e0       ??_C@_0CG@JNNCGPHB@?$CD?5?5?5error?5expected?3?5code?$DN?$CFd?0?5na@ 00000001800051e0     libredefclass008.obj
 0002:00001210       ??_C@_0EB@IMGKPCGE@?$CIstr_obj?5?$DN?5jni?9?$DONewStringUTF?$CIco@ 0000000180005210     libredefclass008.obj
 0002:00001260       ??_C@_0EA@HFOGGBCC@s?2test?2hotspot?2jtreg?2vmTestbase@ 0000000180005260     libredefclass008.obj
 0002:000012a0       ??_C@_05KKCIMGE@error@     00000001800052a0     libredefclass008.obj
 0002:000012b0       ??_C@_0EA@PNBCDMOA@s?2test?2hotspot?2jtreg?2vmTestbase@ 00000001800052b0     libredefclass008.obj
 0002:000012f0       ??_C@_0DI@ILAHDLMP@?$CI?$CKagentThreadProc?$CJ?$CIjvmti_env?0?5a@ 00000001800052f0     libredefclass008.obj
 0002:00001328       ??_C@_0BD@KDBALNLB@JVMTI?5agent?5thread@ 0000000180005328     libredefclass008.obj
 0002:00001340       ??_C@_0BB@NOKBFPFO@java?1lang?1Thread@ 0000000180005340     libredefclass008.obj
 0002:00001354       ??_C@_06FALKBLGB@?$DMinit?$DO@ 0000000180005354     libredefclass008.obj
 0002:00001360       ??_C@_0BG@IKDDPPGD@?$CILjava?1lang?1String?$DL?$CJV@ 0000000180005360     libredefclass008.obj
 0002:00001380       ??_C@_0EB@IFJBFEKC@?$CIthreadClass?5?$DN?5jni_env?9?$DOFindCla@ 0000000180005380     libredefclass008.obj
 0002:000013d0       ??_C@_0GF@FGFIBKKL@?$CIthreadCtor?5?$DN?5jni_env?9?$DOGetMetho@ 00000001800053d0     libredefclass008.obj
 0002:00001438       ??_C@_0DN@NCPDJLOG@?$CIthreadName?5?$DN?5jni_env?9?$DONewStrin@ 0000000180005438     libredefclass008.obj
 0002:00001480       ??_C@_0FE@PFKODBGC@?$CIthreadObject?5?$DN?5jni_env?9?$DONewObj@ 0000000180005480     libredefclass008.obj
 0002:000014e0       ??_C@_0ED@HOBAHHJI@?$CIthreadGlobalRef?5?$DN?5jni_env?9?$DONew@ 00000001800054e0     libredefclass008.obj
 0002:00001530       ??_C@_0FN@HNJJAHFC@jvmti_env?9?$DORunAgentThread?$CIagent@ 0000000180005530     libredefclass008.obj
 0002:00001590       ??_C@_0EA@MOJDNKDF@Debuggee?5status?5sync?5aborted?5be@ 0000000180005590     libredefclass008.obj
 0002:000015d0       ??_C@_0EA@EEOEJAEN@status?5?$DN?5syncDebuggeeStatus?$CIjni@ 00000001800055d0     libredefclass008.obj
 0002:00001610       ??_C@_0BL@JBCFNBMB@nsk_jvmti_resetAgentData?$CI?$CJ@ 0000000180005610     libredefclass008.obj
 0002:00001630       ??_C@_0EL@LPBEELIP@s?2test?2hotspot?2jtreg?2vmTestbase@ 0000000180005630     libredefclass008.obj
 0002:00001680       ??_C@_0CK@JDAMFDMJ@jvmti?9?$DOSetTag?$CIo?0?5tag?$CJ?5?$DN?$DN?5JVMTI_@ 0000000180005680     libredefclass008.obj
 0002:000016b0       ??_C@_0CC@DAMNHKNI@Can?8t?5set?5tag?5?$CFli?5for?5object?5?$CFl@ 00000001800056b0     libredefclass008.obj
 0002:000016d8       ??_C@_0DL@HAJPNKEF@jvmti?9?$DOGetObjectHashCode?$CIo?0?5?$CGha@ 00000001800056d8     libredefclass008.obj
 0002:00001718       ??_C@_0BL@JFPIEOBF@Can?8t?5get?5hash?5object?5?$CFlx?6@ 0000000180005718     libredefclass008.obj
 0002:00001738       ??_C@_0BG@DICPHBKN@setTag?3?5?$CF08x?5?$DM?9?5?$CF?53li@ 0000000180005738     libredefclass008.obj
 0002:00001750       ??_C@_0DH@FCEEBDMJ@?$CIs?5?$DN?5jni?9?$DOGetStringUTFChars?$CIsIn@ 0000000180005750     libredefclass008.obj
 0002:00001788       ??_C@_0BJ@OKKGHDCN@Can?8t?5get?5string?5at?5?$CF?$CDp?6@ 0000000180005788     libredefclass008.obj
 0002:000017a8       ??_C@_0BP@EKFLGGFJ@Can?8t?5get?5string?5at?5?$CF?$CDp?3?5null?6@ 00000001800057a8     libredefclass008.obj
 0002:000017c8       ??_C@_06ICODBHCL@?5?1?1?5?$CFs@ 00000001800057c8     libredefclass008.obj
 0002:000017d0       ??_C@_0DB@KGFPLEGO@?$CIr?5?$DN?5jvmti?9?$DOGetTag?$CIo?0?5?$CGtag?$CJ?$CJ?5?$DN?$DN@ 00000001800057d0     libredefclass008.obj
 0002:00001808       ??_C@_0CO@PDAGBCGJ@Can?8t?5GetTag?5for?5object?5?$CFlx?4?5Re@ 0000000180005808     libredefclass008.obj
 0002:00001838       ??_C@_0CH@HPEODOHC@TEST_BUG?3?5Max?4?5number?5of?5refs?5r@ 0000000180005838     libredefclass008.obj
 0002:00001860       ??_C@_0DI@PHFCABIM@?$CIr?5?$DN?5jvmti?9?$DOGetTag?$CIfrom?0?5?$CGtagFr@ 0000000180005860     libredefclass008.obj
 0002:00001898       ??_C@_0DI@MDEGFNKD@TEST_BUG?3?5Can?8t?5GetTag?5for?5obje@ 0000000180005898     libredefclass008.obj
 0002:000018d0       ??_C@_0DE@MLELJAHM@?$CIr?5?$DN?5jvmti?9?$DOGetTag?$CIto?0?5?$CGtagTo?$CJ?$CJ@ 00000001800058d0     libredefclass008.obj
 0002:00001910       ??_C@_0FK@BIEPFMFP@s?2test?2hotspot?2jtreg?2vmTestbase@ 0000000180005910     libredefclass008.obj
 0002:00001970       ??_C@_0CF@JMMADLFE@?$CFs?3?5Failed?5to?5call?5GetEnv?3?5erro@ 0000000180005970     libredefclass008.obj
 0002:00001998       ??_C@_0DG@LAJPGIIE@?$CIGetPotentialCapabilities?$CJ?5unex@ 0000000180005998     libredefclass008.obj
 0002:000019d0       ??_C@_0CN@LKPEOJPO@?$CIAddCapabilities?$CJ?5unexpected?5er@ 00000001800059d0     libredefclass008.obj
 0002:00001a00       ??_C@_0CN@BCCBOHCH@?$CIGetCapabilities?$CJ?5unexpected?5er@ 0000000180005a00     libredefclass008.obj
 0002:00001a30       ??_C@_0CN@DLBMMHNI@Warning?3?5RedefineClasses?5is?5not@ 0000000180005a30     libredefclass008.obj
 0002:00001a60       ??_C@_0CP@IMINGNLL@?$CISetEventCallbacks?$CJ?5unexpected?5@ 0000000180005a60     libredefclass008.obj
 0002:00001a90       ??_C@_0CO@FDBBPEKA@Warning?3?5Breakpoint?5event?5is?5no@ 0000000180005a90     libredefclass008.obj
 0002:00001ac0       ??_C@_0FC@PKMOONLI@?$CFs?3?5Failed?5to?5get?5the?5method?5ID@ 0000000180005ac0     libredefclass008.obj
 0002:00001b20       ??_C@_0FA@NJGGMIEM@?$CFs?3?5Failed?5to?5get?5the?5method?5ID@ 0000000180005b20     libredefclass008.obj
 0002:00001b70       ??_C@_08EMNENPBA@instance@ 0000000180005b70     libredefclass008.obj
 0002:00001b7c       ??_C@_06GGHJAEBN@static@   0000000180005b7c     libredefclass008.obj
 0002:00001b90       ??_C@_0GL@DIJHFMBD@?$DO?$DO?$DO?$DO?$DO?$DO?$DO?$DO?5?$CD?$CFd?5Invoke?5SetBreakpoi@ 0000000180005b90     libredefclass008.obj
 0002:00001c00       ??_C@_0DC@OFMOJOEC@?$CFs?3?5Failed?5to?5call?5SetBreakpoin@ 0000000180005c00     libredefclass008.obj
 0002:00001c38       ??_C@_0CM@NEGFNKGE@Failed?5to?5enable?5BREAKPOINT?5eve@ 0000000180005c38     libredefclass008.obj
 0002:00001c68       ??_C@_0DE@DFMDMOIM@?$DM?$DM?$DM?$DM?$DM?$DM?$DM?$DM?5?$CD?$CFd?5SetBreakpoint?$CI?$CJ?5is@ 0000000180005c68     libredefclass008.obj
 0002:00001ca0       ??_C@_0CH@CDOJMNAO@JVMTI?5client?5was?5not?5properly?5l@ 0000000180005ca0     libredefclass008.obj
 0002:00001cc8       ??_C@_0DN@HPFPLBDL@?$DO?$DO?$DO?$DO?$DO?$DO?$DO?$DO?5Invoke?5RedefineClasses@ 0000000180005cc8     libredefclass008.obj
 0002:00001d08       ??_C@_0DE@FNJIIKFO@?$CFs?3?5Failed?5to?5call?5RedefineClas@ 0000000180005d08     libredefclass008.obj
 0002:00001d40       ??_C@_0DF@KIBMOCOK@?7For?5more?5info?5about?5this?5error@ 0000000180005d40     libredefclass008.obj
 0002:00001d78       ??_C@_0DC@OOHPOGMA@?$DM?$DM?$DM?$DM?$DM?$DM?$DM?$DM?5RedefineClasses?$CI?$CJ?5is?5s@ 0000000180005d78     libredefclass008.obj
 0002:00001db0       ??_C@_0FM@HFFGHKAC@?$CFs?3?5getResult?3?5Failed?5to?5get?5th@ 0000000180005db0     libredefclass008.obj
 0002:00001e10       ??_C@_0FK@BBPKBAAE@?$CFs?3?5getResult?3?5Failed?5to?5get?5th@ 0000000180005e10     libredefclass008.obj
 0002:00001e70       ??_C@_0JG@COMOAFIA@TEST?5FAILED?3?5Breakpoint?5?$CD?$CFd?5in?5@ 0000000180005e70     libredefclass008.obj
 0002:00001f10       ??_C@_0JD@IOHKAOEA@Check?5?$CD?$CFd?5PASSED?3?5Breakpoint?5in@ 0000000180005f10     libredefclass008.obj
 0002:00001fb0       ??_C@_0HM@MHNDIMMM@TEST?5FAILED?3?5the?5function?5SetBr@ 0000000180005fb0     libredefclass008.obj
 0002:00002040       ??_C@_1EC@JIJBPKFM@?$AAa?$AAp?$AAi?$AA?9?$AAm?$AAs?$AA?9?$AAw?$AAi?$AAn?$AA?9?$AAc?$AAo?$AAr?$AAe@ 0000000180006040     MSVCRT:thread_safe_statics.obj
 0002:00002088       ??_C@_1BK@MGMFAEKH@?$AAk?$AAe?$AAr?$AAn?$AAe?$AAl?$AA3?$AA2?$AA?4?$AAd?$AAl?$AAl@ 0000000180006088     MSVCRT:thread_safe_statics.obj
 0002:000020a8       ??_C@_0BJ@JEBJOJFJ@SleepConditionVariableCS@ 00000001800060a8     MSVCRT:thread_safe_statics.obj
 0002:000020c8       ??_C@_0BJ@PGPPEPCC@WakeAllConditionVariable@ 00000001800060c8     MSVCRT:thread_safe_statics.obj
 0002:000020e8       _pDefaultRawDllMain        00000001800060e8     MSVCRT:dll_dllmain.obj
 0002:000020e8       _pRawDllMain               00000001800060e8     MSVCRT:dll_dllmain.obj
 0002:000020f0       __xmm@ffffffffffffffffffffffffffffffff 00000001800060f0     MSVCRT:utility.obj
 0002:00002100       _load_config_used          0000000180006100     MSVCRT:loadcfg.obj
 0002:00002300       _tls_used                  0000000180006300     MSVCRT:tlssup.obj
 0002:00002328       __volatile_metadata        0000000180006328     <linker-defined>
 0002:000026f8       __rtc_iaa                  00000001800066f8     MSVCRT:initsect.obj
 0002:00002700       __rtc_izz                  0000000180006700     MSVCRT:initsect.obj
 0002:00002708       __rtc_taa                  0000000180006708     MSVCRT:initsect.obj
 0002:00002710       __rtc_tzz                  0000000180006710     MSVCRT:initsect.obj
 0002:00002718       _tls_start                 0000000180006718     MSVCRT:tlssup.obj
 0002:0000271c       _Init_thread_epoch         000000018000671c     MSVCRT:thread_safe_statics.obj
 0002:00002720       _tls_end                   0000000180006720     MSVCRT:tlssup.obj
 0002:00002e74       __IMPORT_DESCRIPTOR_KERNEL32 0000000180006e74     kernel32:KERNEL32.dll
 0002:00002e88       __IMPORT_DESCRIPTOR_VCRUNTIME140 0000000180006e88     vcruntime:VCRUNTIME140.dll
 0002:00002e9c       __IMPORT_DESCRIPTOR_api-ms-win-crt-runtime-l1-1-0 0000000180006e9c     ucrt:api-ms-win-crt-runtime-l1-1-0.dll
 0002:00002eb0       __IMPORT_DESCRIPTOR_api-ms-win-crt-stdio-l1-1-0 0000000180006eb0     ucrt:api-ms-win-crt-stdio-l1-1-0.dll
 0002:00002ec4       __IMPORT_DESCRIPTOR_api-ms-win-crt-string-l1-1-0 0000000180006ec4     ucrt:api-ms-win-crt-string-l1-1-0.dll
 0002:00002ed8       __NULL_IMPORT_DESCRIPTOR   0000000180006ed8     kernel32:KERNEL32.dll
 0003:000000f8       _Init_global_epoch         00000001800080f8     MSVCRT:thread_safe_statics.obj
 0003:00000100       __security_cookie          0000000180008100     MSVCRT:gs_cookie.obj
 0003:00000108       __security_cookie_complement 0000000180008108     MSVCRT:gs_cookie.obj
 0003:00000110       __scrt_native_dllmain_reason 0000000180008110     MSVCRT:utility.obj
 0003:00000118       __isa_available            0000000180008118     MSVCRT:cpu_disp.obj
 0003:0000011c       __isa_enabled              000000018000811c     MSVCRT:cpu_disp.obj
 0003:00000120       __memset_fast_string_threshold 0000000180008120     MSVCRT:cpu_disp.obj
 0003:00000128       __memset_nt_threshold      0000000180008128     MSVCRT:cpu_disp.obj
 0003:00000130       __scrt_ucrt_dll_is_in_use  0000000180008130     MSVCRT:ucrt_stubs.obj
 0003:00000140       g_wrongHeapCallbacks       0000000180008140     libredefclass008.obj
 0003:000001c0       g_szTagInfo                00000001800081c0     libredefclass008.obj
 0003:00002100       g_tagFlags                 000000018000a100     libredefclass008.obj
 0003:000024e8       g_refsToVerifyCnt          000000018000a4e8     libredefclass008.obj
 0003:000024ec       g_fakeUserData             000000018000a4ec     libredefclass008.obj
 0003:000024f0       g_tagVisitCount            000000018000a4f0     libredefclass008.obj
 0003:00003490       g_refsToVerify             000000018000b490     libredefclass008.obj
 0003:0001ab90       g_userDataError            0000000180022b90     libredefclass008.obj
 0003:0001ae88       ?_OptionsStorage@?1??__local_stdio_printf_options@@9@4_KA 0000000180022e88     libredefclass008.obj
 0003:0001b448       _tls_index                 0000000180023448     MSVCRT:tlssup.obj
 0003:0001b450       __scrt_current_native_startup_state 0000000180023450     MSVCRT:utility.obj
 0003:0001b458       __scrt_native_startup_lock 0000000180023458     MSVCRT:utility.obj
 0003:0001b498       __scrt_debugger_hook_flag  0000000180023498     MSVCRT:utility_desktop.obj
 0003:0001b4a0       ?__type_info_root_node@@3U__type_info_node@@A 00000001800234a0     MSVCRT:tncleanup.obj
 0003:0001b4b0       ?_OptionsStorage@?1??__local_stdio_scanf_options@@9@4_KA 00000001800234b0     MSVCRT:default_local_stdio_options.obj
 0003:0001b4b8       __favor                    00000001800234b8     MSVCRT:cpu_disp.obj
 0003:0001b4c0       __dyn_tls_init_callback    00000001800234c0     <common>

 entry point at        0001:000025e0

 Static symbols

 0000:fffda000       .debug$S                   0000000180000000     redefclass008.exp
 0000:fffda000       .debug$S                   0000000180000000     vcruntime:VCRUNTIME140.dll
 0000:fffda000       .debug$S                   0000000180000000     vcruntime:VCRUNTIME140.dll
 0000:fffda000       .debug$S                   0000000180000000     vcruntime:VCRUNTIME140.dll
 0000:fffda000       .debug$S                   0000000180000000     vcruntime:VCRUNTIME140.dll
 0000:fffda000       .debug$S                   0000000180000000     vcruntime:VCRUNTIME140.dll
 0000:fffda000       .debug$S                   0000000180000000     vcruntime:VCRUNTIME140.dll
 0000:fffda000       .debug$S                   0000000180000000     vcruntime:VCRUNTIME140.dll
 0000:fffda000       .debug$S                   0000000180000000     ucrt:api-ms-win-crt-convert-l1-1-0.dll
 0002:ffffc000       .idata$6                   0000000180000000     ucrt:api-ms-win-crt-convert-l1-1-0.dll
 0000:fffda000       .debug$S                   0000000180000000     ucrt:api-ms-win-crt-heap-l1-1-0.dll
 0000:fffda000       .debug$S                   0000000180000000     ucrt:api-ms-win-crt-heap-l1-1-0.dll
 0000:fffda000       .debug$S                   0000000180000000     ucrt:api-ms-win-crt-heap-l1-1-0.dll
 0000:fffda000       .debug$S                   0000000180000000     ucrt:api-ms-win-crt-heap-l1-1-0.dll
 0002:ffffc000       .idata$6                   0000000180000000     ucrt:api-ms-win-crt-heap-l1-1-0.dll
 0000:fffda000       .debug$S                   0000000180000000     ucrt:api-ms-win-crt-runtime-l1-1-0.dll
 0000:fffda000       .debug$S                   0000000180000000     ucrt:api-ms-win-crt-runtime-l1-1-0.dll
 0000:fffda000       .debug$S                   0000000180000000     ucrt:api-ms-win-crt-runtime-l1-1-0.dll
 0000:fffda000       .debug$S                   0000000180000000     ucrt:api-ms-win-crt-runtime-l1-1-0.dll
 0000:fffda000       .debug$S                   0000000180000000     ucrt:api-ms-win-crt-runtime-l1-1-0.dll
 0000:fffda000       .debug$S                   0000000180000000     ucrt:api-ms-win-crt-runtime-l1-1-0.dll
 0000:fffda000       .debug$S                   0000000180000000     ucrt:api-ms-win-crt-runtime-l1-1-0.dll
 0000:fffda000       .debug$S                   0000000180000000     ucrt:api-ms-win-crt-runtime-l1-1-0.dll
 0000:fffda000       .debug$S                   0000000180000000     ucrt:api-ms-win-crt-runtime-l1-1-0.dll
 0000:fffda000       .debug$S                   0000000180000000     ucrt:api-ms-win-crt-runtime-l1-1-0.dll
 0000:fffda000       .debug$S                   0000000180000000     ucrt:api-ms-win-crt-runtime-l1-1-0.dll
 0000:fffda000       .debug$S                   0000000180000000     ucrt:api-ms-win-crt-runtime-l1-1-0.dll
 0000:fffda000       .debug$S                   0000000180000000     ucrt:api-ms-win-crt-runtime-l1-1-0.dll
 0000:fffda000       .debug$S                   0000000180000000     ucrt:api-ms-win-crt-runtime-l1-1-0.dll
 0000:fffda000       .debug$S                   0000000180000000     ucrt:api-ms-win-crt-runtime-l1-1-0.dll
 0000:fffda000       .debug$S                   0000000180000000     ucrt:api-ms-win-crt-runtime-l1-1-0.dll
 0000:fffda000       .debug$S                   0000000180000000     ucrt:api-ms-win-crt-stdio-l1-1-0.dll
 0000:fffda000       .debug$S                   0000000180000000     ucrt:api-ms-win-crt-stdio-l1-1-0.dll
 0000:fffda000       .debug$S                   0000000180000000     ucrt:api-ms-win-crt-stdio-l1-1-0.dll
 0000:fffda000       .debug$S                   0000000180000000     ucrt:api-ms-win-crt-stdio-l1-1-0.dll
 0000:fffda000       .debug$S                   0000000180000000     ucrt:api-ms-win-crt-stdio-l1-1-0.dll
 0000:fffda000       .debug$S                   0000000180000000     ucrt:api-ms-win-crt-stdio-l1-1-0.dll
 0000:fffda000       .debug$S                   0000000180000000     ucrt:api-ms-win-crt-stdio-l1-1-0.dll
 0000:fffda000       .debug$S                   0000000180000000     ucrt:api-ms-win-crt-stdio-l1-1-0.dll
 0000:fffda000       .debug$S                   0000000180000000     ucrt:api-ms-win-crt-stdio-l1-1-0.dll
 0000:fffda000       .debug$S                   0000000180000000     ucrt:api-ms-win-crt-stdio-l1-1-0.dll
 0000:fffda000       .debug$S                   0000000180000000     ucrt:api-ms-win-crt-string-l1-1-0.dll
 0000:fffda000       .debug$S                   0000000180000000     ucrt:api-ms-win-crt-string-l1-1-0.dll
 0000:fffda000       .debug$S                   0000000180000000     ucrt:api-ms-win-crt-string-l1-1-0.dll
 0000:fffda000       .debug$S                   0000000180000000     ucrt:api-ms-win-crt-string-l1-1-0.dll
 0000:fffda000       .debug$S                   0000000180000000     ucrt:api-ms-win-crt-string-l1-1-0.dll
 0000:fffda000       .debug$S                   0000000180000000     ucrt:api-ms-win-crt-string-l1-1-0.dll
 0000:fffda000       .debug$S                   0000000180000000     ucrt:api-ms-win-crt-string-l1-1-0.dll
 0000:fffda000       .debug$S                   0000000180000000     ucrt:api-ms-win-crt-string-l1-1-0.dll
 0000:fffda000       .debug$S                   0000000180000000     kernel32:KERNEL32.dll
 0000:fffda000       .debug$S                   0000000180000000     kernel32:KERNEL32.dll
 0000:fffda000       .debug$S                   0000000180000000     kernel32:KERNEL32.dll
 0000:fffda000       .debug$S                   0000000180000000     kernel32:KERNEL32.dll
 0000:fffda000       .debug$S                   0000000180000000     kernel32:KERNEL32.dll
 0000:fffda000       .debug$S                   0000000180000000     kernel32:KERNEL32.dll
 0000:fffda000       .debug$S                   0000000180000000     kernel32:KERNEL32.dll
 0000:fffda000       .debug$S                   0000000180000000     kernel32:KERNEL32.dll
 0000:fffda000       .debug$S                   0000000180000000     kernel32:KERNEL32.dll
 0000:fffda000       .debug$S                   0000000180000000     kernel32:KERNEL32.dll
 0000:fffda000       .debug$S                   0000000180000000     kernel32:KERNEL32.dll
 0000:fffda000       .debug$S                   0000000180000000     kernel32:KERNEL32.dll
 0000:fffda000       .debug$S                   0000000180000000     kernel32:KERNEL32.dll
 0000:fffda000       .debug$S                   0000000180000000     kernel32:KERNEL32.dll
 0000:fffda000       .debug$S                   0000000180000000     kernel32:KERNEL32.dll
 0000:fffda000       .debug$S                   0000000180000000     kernel32:KERNEL32.dll
 0000:fffda000       .debug$S                   0000000180000000     kernel32:KERNEL32.dll
 0000:fffda000       .debug$S                   0000000180000000     kernel32:KERNEL32.dll
 0000:fffda000       .debug$S                   0000000180000000     kernel32:KERNEL32.dll
 0000:fffda000       .debug$S                   0000000180000000     kernel32:KERNEL32.dll
 0000:fffda000       .debug$S                   0000000180000000     kernel32:KERNEL32.dll
 0000:fffda000       .debug$S                   0000000180000000     kernel32:KERNEL32.dll
 0000:fffda000       .debug$S                   0000000180000000     kernel32:KERNEL32.dll
 0000:fffda000       .debug$S                   0000000180000000     kernel32:KERNEL32.dll
 0000:fffda000       .debug$S                   0000000180000000     kernel32:KERNEL32.dll
 0000:fffda000       .debug$S                   0000000180000000     kernel32:KERNEL32.dll
 0000:fffda000       .debug$S                   0000000180000000     kernel32:KERNEL32.dll
 0000:fffda000       .debug$S                   0000000180000000     kernel32:KERNEL32.dll
 0001:0000127c       addRefToVerify             000000018000227c f   libredefclass008.obj
 0001:000012f0       agentThreadWrapper         00000001800022f0 f   libredefclass008.obj
 0001:000014c8       file_basename              00000001800024c8 f   libredefclass008.obj
 0001:00001af0       startAgentThreadWrapper    0000000180002af0 f   libredefclass008.obj
 0001:00001e1c       syncDebuggeeStatus         0000000180002e1c f   libredefclass008.obj
 0001:000020a4       capture_previous_context   00000001800030a4 f   MSVCRT:gs_report.obj
 0001:00002118       ?__scrt_initialize_thread_safe_statics@@YAHXZ 0000000180003118 f   MSVCRT:thread_safe_statics.obj
 0001:000021e8       ?__scrt_uninitialize_thread_safe_statics@@YAXXZ 00000001800031e8 f   MSVCRT:thread_safe_statics.obj
 0001:00002290       $$000000                   0000000180003290     MSVCRT:amdsecgs.obj
 0001:000022c0       ?dllmain_crt_dispatch@@YAHQEAUHINSTANCE__@@KQEAX@Z 00000001800032c0 f   MSVCRT:dll_dllmain.obj
 0001:00002310       ?dllmain_crt_process_attach@@YAHQEAUHINSTANCE__@@QEAX@Z 0000000180003310 f   MSVCRT:dll_dllmain.obj
 0001:00002428       ?dllmain_crt_process_detach@@YAH_N@Z 0000000180003428 f   MSVCRT:dll_dllmain.obj
 0001:000024ac       ?dllmain_dispatch@@YAHQEAUHINSTANCE__@@KQEAX@Z 00000001800034ac f   MSVCRT:dll_dllmain.obj
 0001:00002ec0       $$000000                   0000000180003ec0     MSVCRT:guard_dispatch.obj
 0001:00002ee0       $$000000                   0000000180003ee0     MSVCRT:guard_xfg_dispatch.obj
 0001:00002ef6       ?fin$0@?0??dllmain_crt_process_attach@@YAHQEAUHINSTANCE__@@QEAX@Z@4HA 0000000180003ef6 f   MSVCRT:dll_dllmain.obj
 0001:00002f0d       ?fin$0@?0??dllmain_crt_process_detach@@YAH_N@Z@4HA 0000000180003f0d f   MSVCRT:dll_dllmain.obj
 0001:00002f26       ?fin$1@?0??dllmain_crt_process_detach@@YAH_N@Z@4HA 0000000180003f26 f   MSVCRT:dll_dllmain.obj
 0001:00002f3a       ?filt$0@?0??dllmain_dispatch@@YAHQEAUHINSTANCE__@@KQEAX@Z@4HA 0000000180003f3a f   MSVCRT:dll_dllmain.obj
 0001:00002f70       __scrt_is_nonwritable_in_current_image$filt$0 0000000180003f70 f   MSVCRT:utility.obj
 0002:000001e0       ?__scrt_initialize_tss_var@@3P6AHXZEA 00000001800041e0     MSVCRT:thread_safe_statics.obj
 0002:00000300       ?opcLengths@@3QBEB         0000000180004300     libredefclass008.obj
 0002:00002030       GS_ExceptionPointers       0000000180006030     MSVCRT:gs_report.obj
 0002:00002728       $unwind$fprintf            0000000180006728     libredefclass008.obj
 0002:00002734       $unwind$printf             0000000180006734     libredefclass008.obj
 0002:00002740       $unwind$?NewObject@JNIEnv_@@QEAAPEAV_jobject@@PEAV_jclass@@PEAU_jmethodID@@ZZ 0000000180006740     libredefclass008.obj
 0002:00002740       $unwind$nsk_lcomplain      0000000180006740     libredefclass008.obj
 0002:00002740       $unwind$nsk_ldisplay       0000000180006740     libredefclass008.obj
 0002:00002748       $unwind$nsk_lvdisplay      0000000180006748     libredefclass008.obj
 0002:00002748       $unwind$_RTC_Initialize    0000000180006748     MSVCRT:initsect.obj
 0002:00002748       $unwind$_RTC_Terminate     0000000180006748     MSVCRT:initsect.obj
 0002:00002748       $unwind$?__scrt_initialize_thread_safe_statics@@YAHXZ 0000000180006748     MSVCRT:thread_safe_statics.obj
 0002:00002754       $unwind$nsk_lvcomplain     0000000180006754     libredefclass008.obj
 0002:0000276c       $unwind$nsk_ltrace         000000018000676c     libredefclass008.obj
 0002:0000276c       $unwind$__report_gsfailure 000000018000676c     MSVCRT:gs_report.obj
 0002:00002774       $unwind$Agent_Initialize   0000000180006774     libredefclass008.obj
 0002:00002774       $unwind$nsk_lvtrace        0000000180006774     libredefclass008.obj
 0002:00002774       $unwind$__raise_securityfailure 0000000180006774     MSVCRT:gs_report.obj
 0002:00002774       $unwind$__scrt_initialize_crt 0000000180006774     MSVCRT:utility.obj
 0002:00002774       $unwind$__scrt_initialize_onexit_tables 0000000180006774     MSVCRT:utility.obj
 0002:00002774       $unwind$__scrt_release_startup_lock 0000000180006774     MSVCRT:utility.obj
 0002:00002774       $unwind$__scrt_uninitialize_crt 0000000180006774     MSVCRT:utility.obj
 0002:00002774       $unwind$_onexit            0000000180006774     MSVCRT:utility.obj
 0002:0000277c       $unwind$nsk_lverify        000000018000677c     libredefclass008.obj
 0002:0000278c       $unwind$nsk_vprintf        000000018000678c     libredefclass008.obj
 0002:0000279c       $unwind$nsk_printf         000000018000679c     libredefclass008.obj
 0002:000027a4       $unwind$?nsk_jni_lverify@@YAHHPEAUJNIEnv_@@HQEBDH1ZZ 00000001800067a4     libredefclass008.obj
 0002:000027b8       $unwind$?nsk_jni_check_exception@@YAHPEAUJNIEnv_@@QEBDH@Z 00000001800067b8     libredefclass008.obj
 0002:000027d4       $unwind$Java_nsk_jvmti_unit_FollowReferences_FollowRefObjects_resetTags 00000001800067d4     libredefclass008.obj
 0002:000027d4       $unwind$addRefToVerify     00000001800067d4     libredefclass008.obj
 0002:000027d4       $unwind$nsk_jvmti_resetAgentData 00000001800067d4     libredefclass008.obj
 0002:000027d4       $unwind$__scrt_initialize_default_local_stdio_options 00000001800067d4     MSVCRT:default_local_stdio_options.obj
 0002:000027d4       $unwind$?dllmain_crt_dispatch@@YAHQEAUHINSTANCE__@@KQEAX@Z 00000001800067d4     MSVCRT:dll_dllmain.obj
 0002:000027d4       $unwind$DllMain            00000001800067d4     MSVCRT:dll_dllmain_stub.obj
 0002:000027d4       $unwind$__GSHandlerCheck   00000001800067d4     MSVCRT:gshandler.obj
 0002:000027d4       $unwind$?__scrt_uninitialize_thread_safe_statics@@YAXXZ 00000001800067d4     MSVCRT:thread_safe_statics.obj
 0002:000027d4       $unwind$__scrt_acquire_startup_lock 00000001800067d4     MSVCRT:utility.obj
 0002:000027d4       $unwind$__scrt_dllmain_after_initialize_c 00000001800067d4     MSVCRT:utility.obj
 0002:000027d4       $unwind$__scrt_dllmain_before_initialize_c 00000001800067d4     MSVCRT:utility.obj
 0002:000027d4       $unwind$__scrt_dllmain_crt_thread_attach 00000001800067d4     MSVCRT:utility.obj
 0002:000027d4       $unwind$__scrt_dllmain_crt_thread_detach 00000001800067d4     MSVCRT:utility.obj
 0002:000027d4       $unwind$__scrt_dllmain_uninitialize_c 00000001800067d4     MSVCRT:utility.obj
 0002:000027d4       $unwind$__scrt_dllmain_uninitialize_critical 00000001800067d4     MSVCRT:utility.obj
 0002:000027d4       $unwind$atexit             00000001800067d4     MSVCRT:utility.obj
 0002:000027dc       $unwind$nsk_jvmti_lverify  00000001800067dc     libredefclass008.obj
 0002:000027f0       $unwind$exitOnError        00000001800067f0     libredefclass008.obj
 0002:00002800       $unwind$Java_nsk_share_jvmti_ArgumentHandler_getAgentOptionsString 0000000180006800     libredefclass008.obj
 0002:00002814       $unwind$Java_nsk_jvmti_unit_FollowReferences_FollowRefObjects_getTag 0000000180006814     libredefclass008.obj
 0002:00002814       $unwind$Java_nsk_share_jvmti_DebugeeClass_checkStatus 0000000180006814     libredefclass008.obj
 0002:00002814       $unwind$agentThreadWrapper 0000000180006814     libredefclass008.obj
 0002:00002824       $unwind$startAgentThreadWrapper 0000000180006824     libredefclass008.obj
 0002:00002840       $unwind$syncDebuggeeStatus 0000000180006840     libredefclass008.obj
 0002:00002840       $unwind$__scrt_dllmain_exception_filter 0000000180006840     MSVCRT:utility.obj
 0002:00002854       $unwind$Java_nsk_share_jvmti_DebugeeClass_resetAgentData 0000000180006854     libredefclass008.obj
 0002:0000285c       $unwind$MA_checkStatus     000000018000685c     libredefclass008.obj
 0002:00002870       $unwind$Java_nsk_jvmti_unit_FollowReferences_FollowRefObjects_setTag 0000000180006870     libredefclass008.obj
 0002:00002888       $unwind$Java_nsk_jvmti_unit_FollowReferences_FollowRefObjects_addRefToVerify 0000000180006888     libredefclass008.obj
 0002:000028a4       $unwind$Java_nsk_jvmti_RedefineClasses_redefclass008_setBreakpoints 00000001800068a4     libredefclass008.obj
 0002:000028bc       $unwind$Java_nsk_jvmti_RedefineClasses_redefclass008_makeRedefinition 00000001800068bc     libredefclass008.obj
 0002:000028c8       $unwind$Java_nsk_jvmti_RedefineClasses_redefclass008_getResult 00000001800068c8     libredefclass008.obj
 0002:000028e0       $unwind$capture_previous_context 00000001800068e0     MSVCRT:gs_report.obj
 0002:000028ec       $unwind$__GSHandlerCheckCommon 00000001800068ec     MSVCRT:gshandler.obj
 0002:000028f8       $xdatasym                  00000001800068f8     MSVCRT:amdsecgs.obj
 0002:000028fc       $unwind$?dllmain_crt_process_attach@@YAHQEAUHINSTANCE__@@QEAX@Z 00000001800068fc     MSVCRT:dll_dllmain.obj
 0002:00002938       $unwind$?fin$0@?0??dllmain_crt_process_attach@@YAHQEAUHINSTANCE__@@QEAX@Z@4HA 0000000180006938     MSVCRT:dll_dllmain.obj
 0002:00002938       $unwind$?fin$0@?0??dllmain_crt_process_detach@@YAH_N@Z@4HA 0000000180006938     MSVCRT:dll_dllmain.obj
 0002:00002938       $unwind$?fin$1@?0??dllmain_crt_process_detach@@YAH_N@Z@4HA 0000000180006938     MSVCRT:dll_dllmain.obj
 0002:00002940       $unwind$?dllmain_crt_process_detach@@YAH_N@Z 0000000180006940     MSVCRT:dll_dllmain.obj
 0002:00002994       $unwind$?dllmain_dispatch@@YAHQEAUHINSTANCE__@@KQEAX@Z 0000000180006994     MSVCRT:dll_dllmain.obj
 0002:000029bc       $unwind$?filt$0@?0??dllmain_dispatch@@YAHQEAUHINSTANCE__@@KQEAX@Z@4HA 00000001800069bc     MSVCRT:dll_dllmain.obj
 0002:000029c4       $unwind$_DllMainCRTStartup 00000001800069c4     MSVCRT:dll_dllmain.obj
 0002:000029d4       $unwind$__scrt_is_nonwritable_in_current_image 00000001800069d4     MSVCRT:utility.obj
 0002:000029f4       $unwind$__scrt_is_nonwritable_in_current_image$filt$0 00000001800069f4     MSVCRT:utility.obj
 0002:000029fc       $unwind$__scrt_fastfail    00000001800069fc     MSVCRT:utility_desktop.obj
 0002:00002a0c       $unwind$__security_init_cookie 0000000180006a0c     MSVCRT:gs_support.obj
 0002:00002a18       $unwind$__isa_available_init 0000000180006a18     MSVCRT:cpu_disp.obj
 0002:00002a28       $xdatasym                  0000000180006a28     MSVCRT:guard_dispatch.obj
 0002:00002a30       $xdatasym                  0000000180006a30     MSVCRT:guard_xfg_dispatch.obj
 0002:00002a40       .edata                     0000000180006a40     redefclass008.exp
 0002:00002a68       rgpv                       0000000180006a68     redefclass008.exp
 0002:00002aac       rgszName                   0000000180006aac     redefclass008.exp
 0002:00002af0       rgwOrd                     0000000180006af0     redefclass008.exp
 0002:00002b12       szName                     0000000180006b12     redefclass008.exp
 0002:00002b24       $N00001                    0000000180006b24     redefclass008.exp
 0002:00002b33       $N00002                    0000000180006b33     redefclass008.exp
 0002:00002b40       $N00003                    0000000180006b40     redefclass008.exp
 0002:00002b77       $N00004                    0000000180006b77     redefclass008.exp
 0002:00002bb5       $N00005                    0000000180006bb5     redefclass008.exp
 0002:00002bf1       $N00006                    0000000180006bf1     redefclass008.exp
 0002:00002c36       $N00007                    0000000180006c36     redefclass008.exp
 0002:00002c73       $N00008                    0000000180006c73     redefclass008.exp
 0002:00002cbb       $N00009                    0000000180006cbb     redefclass008.exp
 0002:00002cfb       $N00010                    0000000180006cfb     redefclass008.exp
 0002:00002d38       $N00011                    0000000180006d38     redefclass008.exp
 0002:00002d73       $N00012                    0000000180006d73     redefclass008.exp
 0002:00002da1       $N00013                    0000000180006da1     redefclass008.exp
 0002:00002dd2       $N00014                    0000000180006dd2     redefclass008.exp
 0002:00002e01       $N00015                    0000000180006e01     redefclass008.exp
 0002:00002e30       $N00016                    0000000180006e30     redefclass008.exp
 0002:00002e65       $N00017                    0000000180006e65     redefclass008.exp
 0002:0000326a       .idata$6                   000000018000726a     kernel32:KERNEL32.dll
 0002:000032ce       .idata$6                   00000001800072ce     vcruntime:VCRUNTIME140.dll
 0002:00003430       .idata$6                   0000000180007430     ucrt:api-ms-win-crt-runtime-l1-1-0.dll
 0002:00003452       .idata$6                   0000000180007452     ucrt:api-ms-win-crt-stdio-l1-1-0.dll
 0002:00003472       .idata$6                   0000000180007472     ucrt:api-ms-win-crt-string-l1-1-0.dll
 0003:00000000       ?codeAttributeName@@3PEBDEB 0000000180008000     libredefclass008.obj
 0003:00000008       ?lineNumberAttributeName@@3PEBDEB 0000000180008008     libredefclass008.obj
 0003:00000010       ?localVarAttributeName@@3PEBDEB 0000000180008010     libredefclass008.obj
 0003:00000018       ?localVarTypeAttributeName@@3PEBDEB 0000000180008018     libredefclass008.obj
 0003:00000020       ?stackMapAttributeName@@3PEBDEB 0000000180008020     libredefclass008.obj
 0003:00000028       ?callBytes@@3PAEA          0000000180008028     libredefclass008.obj
 0003:0000002c       ?allocBytes@@3PAEA         000000018000802c     libredefclass008.obj
 0003:00000030       breakpoints                0000000180008030     libredefclass008.obj
 0003:0001ab94       redefineAttempted          0000000180022b94     libredefclass008.obj
 0003:0001ab98       nsk_context                0000000180022b98     libredefclass008.obj
 0003:0001aba4       redefineSucceed            0000000180022ba4     libredefclass008.obj
 0003:0001aba8       agentFailed                0000000180022ba8     libredefclass008.obj
 0003:0001abac       currentAgentStatus         0000000180022bac     libredefclass008.obj
 0003:0001abb0       context                    0000000180022bb0     libredefclass008.obj
 0003:0001ac68       agentThread                0000000180022c68     libredefclass008.obj
 0003:0001ac70       agentThreadProc            0000000180022c70     libredefclass008.obj
 0003:0001ac78       agentThreadArg             0000000180022c78     libredefclass008.obj
 0003:0001ac80       agent_data                 0000000180022c80     libredefclass008.obj
 0003:0001ac90       jvmti_env                  0000000180022c90     libredefclass008.obj
 0003:0001ac98       jvm                        0000000180022c98     libredefclass008.obj
 0003:0001aca0       jni_env                    0000000180022ca0     libredefclass008.obj
 0003:0001aca8       checkStatus_func           0000000180022ca8     libredefclass008.obj
 0003:0001acb0       ?codeAttributeIndex@@3GA   0000000180022cb0     libredefclass008.obj
 0003:0001acb4       ?lineNumberAttributeIndex@@3GA 0000000180022cb4     libredefclass008.obj
 0003:0001acb8       ?localVarAttributeIndex@@3GA 0000000180022cb8     libredefclass008.obj
 0003:0001acbc       ?localVarTypeAttributeIndex@@3GA 0000000180022cbc     libredefclass008.obj
 0003:0001acc0       ?stackMapAttributeIndex@@3GA 0000000180022cc0     libredefclass008.obj
 0003:0001acc4       ?stackFrameOffset@@3GA     0000000180022cc4     libredefclass008.obj
 0003:0001acc8       ?mode@@3HA                 0000000180022cc8     libredefclass008.obj
 0003:0001accc       ?constantPoolSize@@3GA     0000000180022ccc     libredefclass008.obj
 0003:0001acd0       ?orig@@3PEBEEB             0000000180022cd0     libredefclass008.obj
 0003:0001acd8       ?gen@@3PEAEEA              0000000180022cd8     libredefclass008.obj
 0003:0001ace0       ?inputPos@@3PEAEEA         0000000180022ce0     libredefclass008.obj
 0003:0001ace8       ?endPos@@3PEBEEB           0000000180022ce8     libredefclass008.obj
 0003:0001acf0       ?genPos@@3PEAEEA           0000000180022cf0     libredefclass008.obj
 0003:0001acf8       ?markPos@@3PEAEEA          0000000180022cf8     libredefclass008.obj
 0003:0001ad00       ?constantPool@@3PEAPEADEA  0000000180022d00     libredefclass008.obj
 0003:0001ad08       ?constantPoolCount@@3GA    0000000180022d08     libredefclass008.obj
 0003:0001ad0c       ?zeroBytes@@3PAEA          0000000180022d0c     libredefclass008.obj
 0003:0001ad10       ?codeLength@@3IA           0000000180022d10     libredefclass008.obj
 0003:0001ad18       ?map@@3PEAIEA              0000000180022d18     libredefclass008.obj
 0003:0001ad20       ?widening@@3PEACEA         0000000180022d20     libredefclass008.obj
 0003:0001ad28       redefCls                   0000000180022d28     libredefclass008.obj
 0003:0001ad30       jvmti                      0000000180022d30     libredefclass008.obj
 0003:0001ad38       caps                       0000000180022d38     libredefclass008.obj
 0003:0001ad50       callbacks                  0000000180022d50     libredefclass008.obj
 0003:0001ae90       GS_ExceptionRecord         0000000180022e90     MSVCRT:gs_report.obj
 0003:0001af30       GS_ContextRecord           0000000180022f30     MSVCRT:gs_report.obj
 0003:0001b400       ?g_tss_cv@@3U_RTL_CONDITION_VARIABLE@@A 0000000180023400     MSVCRT:thread_safe_statics.obj
 0003:0001b408       ?g_tss_event@@3PEAXEA      0000000180023408     MSVCRT:thread_safe_statics.obj
 0003:0001b410       ?g_tss_mutex@@3U_RTL_CRITICAL_SECTION@@A 0000000180023410     MSVCRT:thread_safe_statics.obj
 0003:0001b438       ?g_sleep_condition_variable_cs@@3P6AHPEAU_RTL_CONDITION_VARIABLE@@PEAU_RTL_CRITICAL_SECTION@@K@ZEA 0000000180023438     MSVCRT:thread_safe_statics.obj
 0003:0001b440       ?g_wake_all_condition_variable@@3P6AXPEAU_RTL_CONDITION_VARIABLE@@@ZEA 0000000180023440     MSVCRT:thread_safe_statics.obj
 0003:0001b44c       ?__proc_attached@@3HA      000000018002344c     MSVCRT:dll_dllmain.obj
 0003:0001b460       ?is_initialized_as_dll@@3_NA 0000000180023460     MSVCRT:utility.obj
 0003:0001b461       ?module_local_atexit_table_initialized@@3_NA 0000000180023461     MSVCRT:utility.obj
 0003:0001b468       ?module_local_atexit_table@@3U_onexit_table_t@@A 0000000180023468     MSVCRT:utility.obj
 0003:0001b480       ?module_local_at_quick_exit_table@@3U_onexit_table_t@@A 0000000180023480     MSVCRT:utility.obj
